:100000006E2883169B0083161C141A089B0A6A2804
:1000100083169A001C1555309D00AA309D009C1433
:100020009C1810281C119B0A6A2883178001840AD7
:10003000FF3E031D16286A28210820040319A00A80
:100040008030201AA1062019A106A018A106210DB2
:10005000A00DA10D20086A28A601A500FF30A50764
:10006000031CA607031C6A280330A400DF303A20D3
:100070002E28A401E83EA300A409FC30031C432859
:10008000A30703184028A3070000A40F4028231843
:100090004928A31C4D2800004D280800A801A701ED
:1000A0001030A900240DA70DA80D2508A7022608C9
:1000B000031C260FA802031864282508A707260892
:1000C0000318260FA8070310A30DA40DA90B52288F
:1000D00023086A28831383120313080007309F0044
:1000E000850186013C30831685003F3086008113F0
:1000F000003083120120A2002208AE070318AF0AC5
:1001000083169B0183122E0808202F080820203018
:10011000840060301620A03084005030162020303B
:1001200084003030152000300120AE000320AF00E5
:100130000029851430082C20051430082C20851740
:1001400030082C20051730082C20861730082C206A
:10015000061730082C20B00108008310B11A831450
:1001600083188514831C85108310311A8314831817
:100170000514831C05108310B11983148318851787
:10018000831C851383103119831483180517831C6E
:1001900005138310B118831483188617831C8613E4
:1001A00083103118831483180617831C06136430D8
:1001B0002C2008000130B2000C3032020318EF2866
:1001C000AD302E07A00008300318013E2F07A10014
:1001D0001C20AE002108AF00B20A031DDC28CC3081
:1001E000AA000C30AB002E08A3002F08A4002A0898
:1001F000A5002B08A6004E20AC002408AD00080086
:100200002030B100AD200130B200063032020318B8
:100210000F290310B10CAD20B20A031D05290130CE
:10022000B2000630320203181B290310B10DAD20B5
:10023000B20A031D11296430B00099201F30B100AB
:10024000AD200F30B100AD200730B100AD2003303C
:10025000B100AD200130B100AD20B101AD2064305E
:10026000B0009920C8302C20861D3A29EA30A6001B
:1002700060302D20DA202C032D04031D4129851028
:1002800063292C08023A2D04031D4829051063290F
:100290002C08033A2D04031D4F29851363292C08CC
:1002A000043A2D04031D5629051363292C08053A29
:1002B0002D04031D5D29861363292C08063A2D049D
:1002C000031D632906130130A600F4302D20861D7E
:1002D0007529EA30A60060302D20EA30A600603093
:0E02E0002D20EA30A60060302D20312976292D
:02400E00103F61
:00000001FF
